:020000040000FA
:0200000032D0FC
:0200080025D001
:08001800D8CF01F0E8CF00F0A1
:10002000E0CF02F0EACF03F0E9CF04F09EAA02D0BD
:100030009DBA6DD39EA802D09DB862D3FF0004C0C4
:10004000E9FF03C0EAFF02C0E0FF00C0E8FF01C013
:10005000D8FF1000EACF05F0E9CF06F0A1A202D048
:10006000A0B229D0FF00896A8A6A8B6A926A936A71
:10007000800E946E070EC16EC26A096A0A6A0B6A24
:10008000100E156E080ED8EC04F0080EBBEC04F050
:10009000F40EEE6FEF6F00EE00F010EE00F0100EB9
:1000A000156E4DDB03D84EEC04F0FDD7010EB16E9A
:1000B000A282A0821200A192900EB26EB368095083
:1000C000896E0A508A6E0B508B6EEE51EF5D14E014
:1000D000EEC0E9FFEA6A030EEE2702E1F40EEE6FCE
:1000E000EF5000EC03F0EE50100FE826E16EE26AEC
:1000F000EE50E66EEE50E66E210604E2200602E2C5
:1001000021680B96230604E2220602E223680B9282
:10011000250604E2240602E225680B98270604E27D
:10012000260602E227680A90290604E2280602E26F
:1001300029680A942B0604E22A0602E22B680A9830
:100140002D0604E22C0602E22D680A9C2F0604E22A
:100150002E0602E22F68099A310604E2300602E216
:1001600031680996330604E2320602E233680992E6
:1001700006C0E9FF05C0EAFF1100535026E05350C6
:1001800024E00F0EF76E52C0F6FF0800F5501CE099
:10019000F504086EEA6AEFC0E9FF0850EE6E5350AE
:1001A0005324F66E08501524F76E0900F5CF07F0BA
:1001B0000900F550EE6E0750EE6EE95002E0EF6F69
:1001C0001200F40EEF6F12001200270E525C07E6C9
:1001D000086E310E525C03E7085034D21200120050
:1001E0007B0E525C01E01200096A0A6A0B6A896A96
:1001F0008A6A8B6A1200525001EC01F0156E000001
:100200001200800FE84A700CE84A600CE84A500C73
:10021000E84A400CE84A300CE84A200C100CF66E14
:100220000F0EF76E0800F55012001200030E136E49
:10023000F80E146E120013C0EAFF14C0E9FFEE6E50
:10024000EACF13F0E9CF14F0EA50030807E0EA50D0
:10025000040804E0EA50050801E0E8D71200135052
:10026000050849E11450000846E103EEF8F0EE50AD
:100270007D0841E1EE5068083EE1EE5061083BE147
:10028000EE50720838E1EE506D0835E1EE50090885
:1002900032E10000EE5001EC01F00F6E10082BE08F
:1002A000EE500FEC01F027E0E8060F26800E0C6EF2
:1002B000D890EE32D8B0EF8EED52EECF08F0ED5080
:1002C000EE6E08C0EEFF040E116E000E0E6E0C2EC8
:1002D000EFD7096A0A6A0B6A896A8A6A8B6A7CECB8
:1002E00001F0096A0A6A0B6A896A8A6A8B6A020ED5
:1002F000D8EC04F012001200000E126E000E106E08
:1003000092EC01F0400E106E126E92EC01F0800E35
:10031000106E126E92EC01F0C00E106E126E92EC26
:1003200001F012000E50F86E0F50F76E1050F66E7E
:10033000A68EA69CA684A688F29E550EA76EAA0E2F
:10034000A76EA682F28E0A00080E0D6E1150EA6E9C
:100350001250E96E080E0C6EEE50F56E0F000C2E6A
:10036000FBD7A68EA69CA684F29E550EA76EAA0E5B
:10037000A76EA682F28E0D2EEDD7A6940E50F86EC3
:100380000F50F76E1050F66E1150EA6E1250E96E73
:10039000400E0C6E0900F550EE5E03E10C2EFAD70C
:0A03A0001200100EBBEC04F0FCD7B5
:10060000060DF950F350F9260B840B8612000B806F
:100610000B8212000B8A0B8812000A820A801200D9
:100620000A860A8412000A8A0A8812000A8E0A8C34
:1006300012000988098A12000980098612000984BB
:1006400009821200040DF950F350F9260B941200A0
:100650000B9012000B9A12000A9212000A961200D6
:100660000A9A12000A9E12000998120009901200BC
:1006700009941200040DF950F350F9260B8412006E
:100680000B8012000B8A12000A8212000A861200E6
:100690000A8A12000A8E12000988120009801200CC
:1006A00009841200040DF950F350F9260B8612004C
:1006B0000B9212000B9812000A9012000A9412007A
:1006C0000A9812000A9C1200099A12000996120058
:0406D0000992120079
:1007000056A202D09D989BD482D8AD6E98D4ABB23D
:1007100007D0ABB40AD056B40ED0AE505BD88FD44D
:10072000AB98AB88FA0E36D88AD4AE50AB98AB886B
:10073000FC0E30D884D4AE50FB0E2CD880D4C00E22
:1007400094124F0EAF6E240EAC6E900EAB6E566AC6
:10075000516A526A536A506A546A556A09D811D864
:100760009D8A9D889F9A9F98D08EF28CF28E12005F
:10077000000E5A6E5C6E620E5B6E5D6E5690568217
:100780001200000E5E6E606E720E5F6E616E5694A9
:10079000568612009D9856B01BD05CC0EAFF5DC023
:1007A000E9FFEE6E000EEA6205D0720EE96202D039
:1007B00000EE62F0EACF5CF0E9CF5DF05A505C6287
:1007C00004D05B505D6201D0568056929D88120025
:1007D0009D88120056B41AD060C0EAFF61C0E9FFDC
:1007E000EE6E000EEA6205D0820EE96202D000EEE3
:1007F00072F0EACF60F0E9CF61F05E50606204D041
:100800005F50616201D0568456961200120056B2B3
:100810001CD05AC0EAFF5BC0E9FFEECF59F0000ED2
:10082000EA6205D0720EE96202D000EE62F0EACF11
:100830005AF0E9CF5BF05C505A6204D05D505B62C5
:1008400001D05682569059501200000C9D9A56B60F
:100850001DD05EC0EAFF5FC0E9FFEECF58F0000E8A
:10086000EA6205D0820EE96202D000EE72F0EACFB1
:100870005EF0E9CF5FF060505E6204D061505F626D
:1008800001D05686569458509D8A12009D8A000CBD
:1008900056B61200DBDF7EDFFBD7120056B6120021
:1008A000D5DF506E505050AE35D0516E51AC2ED079
:1008B0005150F00BE0082AE05150F00BF00822E113
:1008C0005150F20823E05150F1081CE05150F30858
:1008D00019E05150F00844E05150E84AA6D4E84AE3
:1008E000A4D4E84AA2D4E84AA0D4E84A9ED4E84A6C
:1008F0009CD4E84A9AD4E84A98D4E84AB0D4E84A62
:1009000094D41200546A010E556E1200546A020EFD
:10091000556E120055BE8FD454660FD050C052F0A1
:10092000542A5450555C01E01200546AD90E515CAF
:1009300020E0C90E515C1BE0120050C053F0546A15
:10094000990E515C10E0890E515C0FE0B90E515CBC
:100950000DE0A90E515C0CE0E90E515C0BE01200B9
:10096000800E556E63D4BDEF00F02FD439D443D43C
:100970005CD45BD45AD4506E516A526A5050536E54
:10098000515052648B9C52608B8C00000000000020
:100990000000000000000000523EF2D7532EF0D7B6
:1009A000513EECD78B9C516A526A536A506A1200CE
:1009B000506E516A526A5050536E515052648B8C33
:1009C00052608B9C0000000000000000000000004E
:1009D0000000523EF2D7532EF0D7513EECD78B8C0D
:0A09E000516A526A536A506A12000D
:100F000000000000000000000000000000000000E1
:100F100000000000000000000000000000000000D1
:100F20000000000000000001020304050607080994
:100F30000A0B00000000000000000000000000009C
:100F400000000000000000000000000000000000A1
:100F50000000000000000000000000000000000091
:100F60000000000000000000000000000000000081
:100F70000000000000000000000000000000000071
:1010000000002A00450060007B009600B100CC0083
:10101000E70002011D01380153016E018901A4019D
:10102000BF01DA01F50110022B02460261027C02C7
:101030009702B202CD02E80203031E0339035403F0
:101040006F038903A403BF03DA03F50310042B0421
:10105000460461047C049704B204CD04E80403054B
:101060001E05390554056F058A05A505C005DB0574
:10107000F60511062C06470662067D069806B3069D
:10108000CE06E90604071F073A07550770078B07C6
:10109000A607C107DC07F70712082D0848086308F0
:1010A0007E089908B408CF08EA08050920093B0919
:1010B000560971098C09A709C209DD09F809130A43
:1010C0002D0A480A630A7E0A990AB40ACF0AEA0A74
:1010D000050B200B3B0B560B710B8C0BA70BC20B9C
:1010E000DD0BF80B130C2E0C490C640C7F0C9A0CC6
:1010F000B50CD00CEB0C060D210D3C0D570D720DEF
:1011000000002A00450060007B009600B100CC0082
:10111000E70002011D01380153016E018901A4019C
:10112000BF01DA01F50110022B02460261027C02C6
:101130009702B202CD02E80203031E0339035403EF
:101140006F038903A403BF03DA03F50310042B0420
:10115000460461047C049704B204CD04E80403054A
:101160001E05390554056F058A05A505C005DB0573
:10117000F60511062C06470662067D069806B3069C
:10118000CE06E90604071F073A07550770078B07C5
:10119000A607C107DC07F70712082D0848086308EF
:1011A0007E089908B408CF08EA08050920093B0918
:1011B000560971098C09A709C209DD09F809130A42
:1011C0002D0A480A630A7E0A990AB40ACF0AEA0A73
:1011D000050B200B3B0B560B710B8C0BA70BC20B9B
:1011E000DD0BF80B130C2E0C490C640C7F0C9A0CC5
:1011F000B50CD00CEB0C060D210D3C0D570D720DEE
:1012000000002A00450060007B009600B100CC0081
:10121000E70002011D01380153016E018901A4019B
:10122000BF01DA01F50110022B02460261027C02C5
:101230009702B202CD02E80203031E0339035403EE
:101240006F038903A403BF03DA03F50310042B041F
:10125000460461047C049704B204CD04E804030549
:101260001E05390554056F058A05A505C005DB0572
:10127000F60511062C06470662067D069806B3069B
:10128000CE06E90604071F073A07550770078B07C4
:10129000A607C107DC07F70712082D0848086308EE
:1012A0007E089908B408CF08EA08050920093B0917
:1012B000560971098C09A709C209DD09F809130A41
:1012C0002D0A480A630A7E0A990AB40ACF0AEA0A72
:1012D000050B200B3B0B560B710B8C0BA70BC20B9A
:1012E000DD0BF80B130C2E0C490C640C7F0C9A0CC4
:1012F000B50CD00CEB0C060D210D3C0D570D720DED
:1013000000002A00450060007B009600B100CC0080
:10131000E70002011D01380153016E018901A4019A
:10132000BF01DA01F50110022B02460261027C02C4
:101330009702B202CD02E80203031E0339035403ED
:101340006F038903A403BF03DA03F50310042B041E
:10135000460461047C049704B204CD04E804030548
:101360001E05390554056F058A05A505C005DB0571
:10137000F60511062C06470662067D069806B3069A
:10138000CE06E90604071F073A07550770078B07C3
:10139000A607C107DC07F70712082D0848086308ED
:1013A0007E089908B408CF08EA08050920093B0916
:1013B000560971098C09A709C209DD09F809130A40
:1013C0002D0A480A630A7E0A990AB40ACF0AEA0A71
:1013D000050B200B3B0B560B710B8C0BA70BC20B99
:1013E000DD0BF80B130C2E0C490C640C7F0C9A0CC3
:1013F000B50CD00CEB0C060D210D3C0D570D720DEC
:1014000000002A00450060007B009600B100CC007F
:10141000E70002011D01380153016E018901A40199
:10142000BF01DA01F50110022B02460261027C02C3
:101430009702B202CD02E80203031E0339035403EC
:101440006F038903A403BF03DA03F50310042B041D
:10145000460461047C049704B204CD04E804030547
:101460001E05390554056F058A05A505C005DB0570
:10147000F60511062C06470662067D069806B30699
:10148000CE06E90604071F073A07550770078B07C2
:10149000A607C107DC07F70712082D0848086308EC
:1014A0007E089908B408CF08EA08050920093B0915
:1014B000560971098C09A709C209DD09F809130A3F
:1014C0002D0A480A630A7E0A990AB40ACF0AEA0A70
:1014D000050B200B3B0B560B710B8C0BA70BC20B98
:1014E000DD0BF80B130C2E0C490C640C7F0C9A0CC2
:1014F000B50CD00CEB0C060D210D3C0D570D720DEB
:1015000000002A00450060007B009600B100CC007E
:10151000E70002011D01380153016E018901A40198
:10152000BF01DA01F50110022B02460261027C02C2
:101530009702B202CD02E80203031E0339035403EB
:101540006F038903A403BF03DA03F50310042B041C
:10155000460461047C049704B204CD04E804030546
:101560001E05390554056F058A05A505C005DB056F
:10157000F60511062C06470662067D069806B30698
:10158000CE06E90604071F073A07550770078B07C1
:10159000A607C107DC07F70712082D0848086308EB
:1015A0007E089908B408CF08EA08050920093B0914
:1015B000560971098C09A709C209DD09F809130A3E
:1015C0002D0A480A630A7E0A990AB40ACF0AEA0A6F
:1015D000050B200B3B0B560B710B8C0BA70BC20B97
:1015E000DD0BF80B130C2E0C490C640C7F0C9A0CC1
:1015F000B50CD00CEB0C060D210D3C0D570D720DEA
:1016000000002A00450060007B009600B100CC007D
:10161000E70002011D01380153016E018901A40197
:10162000BF01DA01F50110022B02460261027C02C1
:101630009702B202CD02E80203031E0339035403EA
:101640006F038903A403BF03DA03F50310042B041B
:10165000460461047C049704B204CD04E804030545
:101660001E05390554056F058A05A505C005DB056E
:10167000F60511062C06470662067D069806B30697
:10168000CE06E90604071F073A07550770078B07C0
:10169000A607C107DC07F70712082D0848086308EA
:1016A0007E089908B408CF08EA08050920093B0913
:1016B000560971098C09A709C209DD09F809130A3D
:1016C0002D0A480A630A7E0A990AB40ACF0AEA0A6E
:1016D000050B200B3B0B560B710B8C0BA70BC20B96
:1016E000DD0BF80B130C2E0C490C640C7F0C9A0CC0
:1016F000B50CD00CEB0C060D210D3C0D570D720DE9
:1017000000002A00450060007B009600B100CC007C
:10171000E70002011D01380153016E018901A40196
:10172000BF01DA01F50110022B02460261027C02C0
:101730009702B202CD02E80203031E0339035403E9
:101740006F038903A403BF03DA03F50310042B041A
:10175000460461047C049704B204CD04E804030544
:101760001E05390554056F058A05A505C005DB056D
:10177000F60511062C06470662067D069806B30696
:10178000CE06E90604071F073A07550770078B07BF
:10179000A607C107DC07F70712082D0848086308E9
:1017A0007E089908B408CF08EA08050920093B0912
:1017B000560971098C09A709C209DD09F809130A3C
:1017C0002D0A480A630A7E0A990AB40ACF0AEA0A6D
:1017D000050B200B3B0B560B710B8C0BA70BC20B95
:1017E000DD0BF80B130C2E0C490C640C7F0C9A0CBF
:1017F000B50CD00CEB0C060D210D3C0D570D720DE8
:1018000000002A00450060007B009600B100CC007B
:10181000E70002011D01380153016E018901A40195
:10182000BF01DA01F50110022B02460261027C02BF
:101830009702B202CD02E80203031E0339035403E8
:101840006F038903A403BF03DA03F50310042B0419
:10185000460461047C049704B204CD04E804030543
:101860001E05390554056F058A05A505C005DB056C
:10187000F60511062C06470662067D069806B30695
:10188000CE06E90604071F073A07550770078B07BE
:10189000A607C107DC07F70712082D0848086308E8
:1018A0007E089908B408CF08EA08050920093B0911
:1018B000560971098C09A709C209DD09F809130A3B
:1018C0002D0A480A630A7E0A990AB40ACF0AEA0A6C
:1018D000050B200B3B0B560B710B8C0BA70BC20B94
:1018E000DD0BF80B130C2E0C490C640C7F0C9A0CBE
:1018F000B50CD00CEB0C060D210D3C0D570D720DE7
:1019000000002A00450060007B009600B100CC007A
:10191000E70002011D01380153016E018901A40194
:10192000BF01DA01F50110022B02460261027C02BE
:101930009702B202CD02E80203031E0339035403E7
:101940006F038903A403BF03DA03F50310042B0418
:10195000460461047C049704B204CD04E804030542
:101960001E05390554056F058A05A505C005DB056B
:10197000F60511062C06470662067D069806B30694
:10198000CE06E90604071F073A07550770078B07BD
:10199000A607C107DC07F70712082D0848086308E7
:1019A0007E089908B408CF08EA08050920093B0910
:1019B000560971098C09A709C209DD09F809130A3A
:1019C0002D0A480A630A7E0A990AB40ACF0AEA0A6B
:1019D000050B200B3B0B560B710B8C0BA70BC20B93
:1019E000DD0BF80B130C2E0C490C640C7F0C9A0CBD
:1019F000B50CD00CEB0C060D210D3C0D570D720DE6
:1020000001000100010001000100010001000100C8
:1020100001000100010001000100010001000100B8
:1020200001000100010001000100010001000100A8
:102030000100010001000100010001000100010098
:020000040030CA
:03000100260A00CC
:02000500018177
:060008000FC00FE00F40E5
:00000001FF
